:103800000C942A1C0C94451C0C94451C0C94451CCF
:103810000C94451C0C94451C0C94451C0C94451CA4
:103820000C94451C0C94451C0C94451C0C94451C94
:103830000C94451C0C94451C0C94451C0C94451C84
:103840000C94451C0C94451C0C94451C0C94451C74
:103850000C94451C11241FBECFE5D4E0DEBFCDBFC4
:1038600010E0A0E6B0E0EAEEFEE302C005900D92A3
:10387000A036B107D9F711E0A0E6B0E001C01D9273
:10388000A43AB107E1F70C94381F0C94001C0F9276
:10389000AF93BF93CF93DF93EF93FF93FC01EA01C4
:1038A000DB01C895099231961197D9F7FF91EF91F5
:1038B000DF91CF91BF91AF910F9008950F921F921A
:1038C0000F93AF93BF93CF93DF93EF93FF93FC01DD
:1038D000EA01DB010990199001E043D0329612977A
:1038E000C9F7FC0103E03DD005E03BD0FF91EF912B
:1038F000DF91CF91BF91AF910F911F900F900895DD
:103900000F931F93EF93FF93FC0103E02AD000E88D
:1039100010E0E00FF11FE617F707B9F7FF91EF91FD
:103920001F910F9108950F930F9222D0082E09E056
:1039300018D00F900F9108950F930F92EF93FF936C
:1039400017D0FC0160935700C895802DFF91EF912F
:103950000F900F9108950F930BD001E102D00F91BA
:103960000895E199FECF00935700E895FFFF00000E
:103970000091570000FDFCCF089587E089B98AB116
:1039800088618AB908958AB1877E8AB908958CB909
:103990005E9BFECF5E9A08958CB1992708958BB1F6
:1039A0009927807890700895EF92FF920F931F935C
:1039B000CF93DF937B01C0E0D0E0C617D70770F448
:1039C0008C010E94CF1C8823E1F30E94CC1CF801DB
:1039D00081938F012196CE15DF0598F381E090E069
:1039E000DF91CF911F910F91FF90EF900895EF928B
:1039F000FF920F931F93CF93DF937C018B01C0E065
:103A0000D0E0C017D10738F4F70181917F010E94FF
:103A1000C71C2196F6CF81E090E0DF91CF911F91F6
:103A20000F91FF90EF90089540E050E0481759073C
:103A300050F422E537E000002150304037FFFBCF43
:103A40004F5F5F4FF3CF08950E94C31C0E94000098
:103A500008950E94CF1C8823E1F30E94CC1C803281
:103A600019F481E090E0089585E10E94C71C80E090
:103A700090E0089590E0282F33272138310589F010
:103A80002238310524F42038310549F00DC02238A0
:103A9000310549F02839310539F493E005C092E049
:103AA00003C091E001C092E1892F9927089540E079
:103AB00050E06091A0007091A10046175707D0F424
:103AC0002091A2013091A301E2EAF0E03FBB2EBBBE
:103AD0002F5F3F4F80818DBBE29AE19AE199FECF43
:103AE0004F5F5F4F31964617570780F33093A3011E
:103AF0002093A201089540E050E06091A0007091F1
:103B0000A10046175707B0F42091A2013091A301FC
:103B1000E2EAF0E03FBB2EBB2F5F3F4FE09A8DB350
:103B200081934F5F5F4F46175707A0F33093A30170
:103B30002093A2010895CF93DF93C0E0D0E080915D
:103B4000A0009091A100C817D907A0F4CE018E550E
:103B50009F4F2091A2013091A301220F331FAC018E
:103B600060E870E0C9018C0F9D1F0E945E1CC05868
:103B7000DF4FE5CF0E94AB1CDF91CF91089580917C
:103B8000A2019091A30142EA50E06091A0007091DF
:103B9000A100880F991F0E94471C0895CF93C0E091
:103BA00069E081E090E00E949C1C992784FF03C09B
:103BB0008F7E0E94931C0E94CF1C8823E1F30E94F9
:103BC000CC1C9927823591051CF5803591050CF0A8
:103BD0005CC08134910509F462C0823491057CF4A3
:103BE00081339105B1F18233910524F4C09709F432
:103BF0004CC038C18034910509F438C133C18234D6
:103C0000910509F45FC08534910509F45EC02AC1AD
:103C10008635910509F4F1C0873591054CF482355C
:103C2000910509F45FC08535910509F469C01AC191
:103C30008437910509F4A4C0853791052CF48436A6
:103C4000910509F476C00EC18537910509F4C5C008
:103C500009C10E94291D882309F4ADCF84E10E9487
:103C6000C71C81E40E94C71C86E50E94C71C82E530
:103C70000E94C71C80E20E94C71C83E50E94C71CEB
:103C800084E50E94C71C8BE406C00E94291D88237E
:103C900009F491CF84E10E94C71C80E1E4C061E097
:103CA00070E080E690E00E94D41C0E94291D8823C9
:103CB00009F481CF84E10E94C71C809160000E94BA
:103CC0003A1DE9CF64E170E008C061E070E080E691
:103CD00090E00E94D41C64E070E080E690E00E94D6
:103CE000D41CD3CF0E94291D882309F464CF60E03F
:103CF00070E480E090E00E94801C0E94AB1CCACF60
:103D000062E070E080E690E00E94D41C0E94291DD1
:103D1000882309F450CF2091600080916100992799
:103D2000982F8827820F911D9093A3018093A20161
:103D3000B1CF63E070E080E690E00E94D41C209157
:103D40006100809160009927982F8827820F911D2C
:103D50009093A1008093A000BC0182EA90E00E94B1
:103D6000D41C0E94291D882309F425CF809162006C
:103D7000863419F40E949B1D8DCF0E94571D8ACF57
:103D800063E070E080E690E00E94D41C2091610026
:103D9000809160009927982F8827820F911D90931A
:103DA000A1008093A0000E94291D882309F403CF5D
:103DB00080916200863419F40E94BF1D02C00E94E7
:103DC0007B1D84E10E94C71C6091A0007091A1003E
:103DD00082EA90E00E94F71C60CF0E94291D882390
:103DE00009F4E9CE84E10E94C71C8EE10E94C71C41
:103DF00084E90E94C71C83E04ECF64E070E080E657
:103E000090E00E94D41C0E94291D882309F4D3CE7F
:103E100084E10E94C71C80916000803531F480915C
:103E20006100882361F4C82F17C0883531F4809170
:103E30006100883061F4C3E00FC0803531F48091B7
:103E40006100883049F4C2E007C0883529F48091C8
:103E50006100882309F4C1E069E08C2F99270E9452
:103E60009C1C19CF85E10E94C71CA5CECF91089557
:103E7000CFE5D4E0DEBFCDBFCEE1F894AEEFB1E048
:103E80000E946C1F802D843B71F4AFEFB1E00E9463
:103E90006C1F802D833C39F4ADEFB1E00E946C1FA4
:103EA000802D992781BF0E94BD1C0E94CC1C84E6F6
:103EB00090E00E94141D0E94CF1C882319F00E94DC
:103EC000CE1D04C0C150C8BBCC2389F70E94241D5D
:103ED00080E090E00C94741FE199FECFBFBBAEBBB5
:0A3EE000E09A11960DB20895FFCF8D
:0400000300003800C1
:00000001FF
